:4000000000080020110000006D0100006D01000010B500F0E1FF00F0F1F900F0AFF8C04610B50B4C11232360182000F023FFC022D200084B1A60084A084B1A600422084B69
:400040001A603C32074B1A600023236010BDC046300010400003014040FF008000000140280003400001014010B572B6EE221202084B1A60FF22084B1A60F33A074B1A601D
:4000800090221201064B1A603622064B1A60FFF7C7FF10BD00010240000302400001044008010440080304400000000000000000000000000000000000000000000000009B
:4000C0000000000000000000000000000000000000000000000000000000000000000000000000000000000000000000000000000000000000000000000000000000000000
:4001000010B5064C2378002B07D1054B002B02D0044800E000BF0123237010BDF8000020000000004C160000084B10B5002B03D00749084800E000BF07480368002B00D1C9
:4001400010BD064B002BFBD09847F9E700000000FC0000204C160000700000200000000010B562B600F0AEFBFEE7C04610B501F02BFA03680C2B00D1FEE7FEE770B50F4EA3
:400180000F4D13E029686B68AC68002202E001C901C30432A242FAD1E868002202E0002102C304328242FAD11035013E002EE9D101F010FAFFF7D4FFFEE7C04601000000E6
:4001C000E016000010B5114A136801218B43136000230AE0032B03D89A000D49505800E00C4899000C4A88500133182BF2D9FFF73BFF0A4B1B68002B02D10022074B1A602C
:40020000024A116801230B43136010BD00001040000000006D0100000000002068000020002306E04218013A12789B189BB2013989B20029F6D1584280B270470047C04684
:4002400010B58022024B1A6000F0A2FE10BDC04668000020F0B583B00D006B469E1DDA8001230B7048701400AA70130ACB70171DB9B22800FFF7D4FFE855631D000AE8544A
:40028000A31D1722EA540734A1B296233200280000F0CCFB03B0F0BD70B505000E001400002802D0002000F0E3FD002005E0013CAB19E3181B781818C0B2002CF7D170BDC2
:4002C00010B50C2864D88000404B1B589F468B06591A8B01FF2292019446634401225CE08B06591A8B013A4A94466344042254E08B06591A8B01374A9446634402224CE071
:400300008B06591A8B01344A94466344042244E08B06591A8B01314A9446634401223CE08B06591A8B012E4A94466344012234E08B06591A8B012B4A9446634402222CE0A3
:400340008B06591A8B01284A94466344022224E08B06591A8B01254A9446634402221CE08B06591A8B01224A94466344042214E08B06591A8B011F4A9446634401220CE012
:400380008B06591A8B011C4A94466344042204E0002000F06DFD02220023012A02D11878C0B200E00020022A03D11978587800020843042A09D11A785878000210439A787C
:4003C00012041043DB781B06184310BD50160000C13F0000C53F0000C93F0000D03F0000D13F0000D63F0000D23F0000D43F0000D83F0000DC3F0000E03F000010B50D4BC0
:400400001B68DB0602D400220B4B1A600A4B1B68802B0ED10022084B1A6000210220FFF74FFF002805D000210220FFF749FFFFF705FF10BD540003406800002070B505002A
:4004400001000320FFF73CFF441CA40129000420FFF736FF241829000320FFF731FF421C92010023002608E01078411EC9B2FD2900D801261B18DBB20132A242F4D35B4218
:40048000DCB229000120FFF71BFF844203D1002E03D1062002E0062000E0002070BDC046F0B55F4656464D464446F0B4CD4CA544050000F069FA62B600239A4600270A24E6
:4004C0009946002D01D1FF2300E02B00C64A02A98C4662449621490052A800F071FA002D01D0013CE4B2002C01D00028E9D1002800D0D7E1BC4B02AA944663441B88062B01
:4005000024D952AA1278012A22D152A9CA78120289780A439146110007329A421AD896235B009A4218D84A1D52AB9E5C3202081D1E5C164306315B5C172B0FD181B252A8E5
:40054000FFF76EFE86420BD100260AE0042608E0042606E0032604E0032602E0042600E00826002E00D04BE152AB1A7993465A781300313BD9B20A2900D901E18B009B4927
:40058000CB589F46012F00D03CE14B46002B00D03BE10020FFF752FF4342434152AA1371012278E1012F00D032E14B46012B00D031E15B46002B00D030E18D4B1B681B68C5
:4005C0009A0BD2B2934503D19B09FF22134005E0934501D9002301E080235B0052AA13711B0A5371FF2393710023D371042252E1342A0DD1012F00D013E14B46032B00D067
:4006000012E10C32002107A801F013F840239A46012F00D00BE14B46022B00D80AE107A85044DA1E4821FF3102AB9C46614400F0F7FF4B4653449BB2432B00D0FDE052AA93
:4006400093791B02527913439A46FF2B00D90A26002E00D0F8E05B461802504480B2644B1B681A6893099BB2920601D001339BB2834200D9ECE007A900F090FA002800D1B2
:40068000EDE000239A46403399460A26002202E1012F00D104E104260022FCE0012F00D0E3E04B46534496225200934200D9DFE007A850444A4653A900F0B2FF53464B44DB
:4006C0009BB29A460022E6E04B46002B00D0D2E004AA484B03CB03C253AA04AB03CB03C200239A4601270822D5E0012F00D0C5E04B46032B00D0C4E052AA93791B025279C2
:40070000134398465B461902414489014346FF2B00D90A26002E00D0B6E040220020FFF7BBFD030001905A461202424492B25946002911D1FF2A0FD10520FFF7C1FDC0B22A
:40074000019B1B1ADBB2984600210620FFF7B8FDC3B24246D31ADBB25B4252AA1371012299E00020FFF76AFE002802D18022224B1A6000F021F900F00BFC042600228AE062
:400780001E4B1E68002E00D180E0012F00D080E002AB1A704A465A8053AB03930C22002104A800F046FF04AB9B4653AA0692190002A8B0475B469A882623FF339A4203D951
:4007C00053AB0699994207D0069B002B01D1002A05D1049BDEB25EE00E2600225BE00E26002258E084FDFFFF6E0200008416000074000020B01600006800002014010020E0
:40080000002248E00426002245E00426002242E0042600223FE0042600223CE00426002239E00426002236E00426002233E00426002230E0042600222DE000239A4640336B
:4008400099460326002226E040239946002222E000239A46403399460A2600221BE000239A4640339946002215E00426002212E0032600220FE0042600220CE004260022D8
:4008800009E00426002206E0002204E00526002201E00526002252A93000FFF7DBFC01E000239A46002D00D10BE6012F00D108E69F239B009D443CBC90469946A246AB461E
:4008C000F0BDC04670B50020FFF7B8FD002801D0062400E00024154D2B681A68C03AC0210020FFF7D9FC6B681B78C01AC0B24042C0B2834204D10D4B1B681B68002B02D155
:40090000002000F0B5FA0A4B1B68402B01D0002C05D00022064B1A600020FFF7C1FD1420FFF7BEFDFFF78CFC70BDC04674000020680000200F4B1B685B0619D50E4B1B6868
:40094000DB060BD50D4B1B68002B11D00C4A136000230C4A1360094A136009E0094B1A68074B1B689A4203D0054B1A68054B1A607047C0464C0F0640640006401801002034
:40098000C0010020B001002010B5094C201D402100F082F820004430002100F05FF8054800F074FB0023236000F04AFB10BDC046180100203509000010B500F051FB10BDC8
:4009C000F8B507000E001500002825D0002925D09A00D3185C001BE0114B1B78DB0613D5104B1A682A8000220D490A701A602B88321C9E4200D91A1C92B20B490431380069
:400A000000F00EFE00200AE0012000F0CDFA013C002CE1D1102002E0012000E00120F8BDB8010020BC0100201801002070B50C0000280DD000290DD01180074D2B00443322
:400A40000A000100180000F0EBFD2C60002002E0012000E0012070BD1801002070B504000D0000280ED0052000F0EEF9064B1C60064B1D600023064A1360064A13600520C4
:400A800000F0D8F970BDC046CC010020C0010020B0010020B401002070B504000D0000280CD0052000F0D0F9054B1C60054B1D600022054B1A60052000F0BCF970BDC04634
:400AC000C8010020C4010020BC010020074B1B68074A1360074B1B68DB0FDB075360064B1B689B001833936000207047280003409C01002030000340080F034010B5124BC3
:400B00009B68302B08D1104B1B689A0704D11B0903221340012B15D0022000F079F90A4B9B68302B02D0302000F0A4F900F04EF9002000F05DF905490B6830229343203AB7
:400B400013430B60002010BD9C0100202800034010B5104B9868302807D11B689A0704D11B0903221340012B11D0302801D000F081F9084C03202368184000F039F9064B4D
:400B800022681A606368002B01D100F029F9002010BDC0469C01002028000340F0B5474680B496B00500002315931493FF2800D9F5E0002900D1F2E0402204A800F030FD4D
:400BC000022300200021002408E09A0002AE9259002A02D0891810431C000133112BF4D9002903D1002803D1002602E0002600E00126002E06D0A30002AA9F58002202A9C0
:400C00005A5000E00027694B02933F230393684B02AA1A606749684A1160C0461B681B0F1B07F0221206934204D1614B1B68FF2213400DE05E4B1B681B0F1B07A02212068B
:400C4000934204D05A4B1B68FF22134000E000231593159B002B00D0A3E000F0CFF90190FFF734FF1490149B002B02D1FFF746FF1590159B002B25D1504A029202992A04EB
:400C80000A4302924A4A02A911604D484A490860C0461268120F1207F02109068A4204D1434B1B68FF2213400BE0414A1268120F1207A02109068A4203D03D4B1B68FF224E
:400CC00013401593159B9846002B59D1002E57D04022002104A800F0ACFCA40002ABE750324B02933F230393314B02AA1A603149314A1160C0461B681B0F1B07F022120661
:400D0000934205D12A4B1B68FF221A4090460CE0274B1B681B0F1B07A0221206934204D0234B1B68FF221A40904643461593159B002B25D1234A0292029A2D04154302950E
:400D40001B4A02A9116020481B490860C0461268120F1207F02109068A4204D1144B1B68FF2213400BE0124A1268120F1207A02109068A4203D00E4B1B68FF22134015938B
:400D8000149B002B07D1FFF7E3FE1490149B002B01D0149B1593019800F034F901E004231593159816B004BC9046F0BDB6D70000080010400400008004001040B6D800009D
:400DC00005000080B6D9000006000080034A1368802109060B4313607047C04630000340024A13685B005B08136070473000034010B5040000F002F9044A136803218B435F
:400E00000C401C43146000F0FDF810BD2800034070B5040000F0F2F805490A680C25AA43A3002C001C4014430C6000F0EBF870BD280003401F2318401E3B8340014A1360C8
:400E40007047C04600E100E01F2318401E3B8340014A13607047C04680E100E01F2318401E3B8340014A13607047C04680E200E001BE7047F8B50400182803D0202801D0BC
:400E800030283CD100F0BAF805001F4A136807218B4313601D4BE3181B78DBB21C4A13601C4A13688B4313601B4803687F22934319001A4BE3181B7813400B4303603220B4
:400EC00000F092F8182C16D90F4E33680727BB431A0023001C3B9B083B4013433360322000F082F83268BA432300183B9B083C001C4014433460280000F084F802E0002001
:400F0000FFF7B6FFF8BDC046080F0340CDF1FF0F0C0F0340100F0340180F0340B4F1FF0F70B504000D00082802D90020FFF7A0FF1034A40080239B059C4664442068256090
:400F400070BDC04670B504000E00032902D90020FFF78EFF082C02D90020FFF789FF03252540ED00063500F049F8A408A400074B9C46644421680323AB4099430B003100EC
:400F8000A9401943216000F03DF870BD00E400E0034A13681B041B0C02490B43136070470CED00E00400FA0510B5040006E0084B586800F019F8074B9C46644480231B0249
:400FC0009C42F4D8024B9868604300F00DF810BD7C0000200080FFFF014A024B1A6070476588EDAC380003400230800804D0C0460138FDD1C046C046C0467047EFF31080DB
:4010000072B6704780F310887047C04610B50520FFF710FF10BDC04610B500F0BDF810BD10B500F057F810BD10B5044A1368802109060B431360FFF7E9FF10BD000006404F
:4010400010B5064B1B78002B04D1FFF7E9FF0122024B1A70FFF7E8FF10BDC046A801002010B50520FFF7F0FEFFF7D6FF054A13685B005B0813600022034B1A600520FFF7DD
:40108000EDFE10BD00000640880F0640014B58607047C046A80100200A4B1B68DB050DD5094B1B685B0409D4064B1968074A0A401A601A68802149000A431A600222044B91
:4010C0001A6070470000064060000640FFFEFFFF6C00064010B500241A4B1C601A4A1B4B1A601B4B1B4A13601B4A14601B491C4A11601C4A13601C4B1C600520FFF7A4FE4D
:4011000003210520FFF71EFF18490520FFF708FF174B1C604C22FF32164B1A60164B1C60164B1C60164B1C603C3AFF3A154B1A70154B1C70154B1C60154B1C60154B1C70B8
:4011400010BDC0460000064088080040600006400701008000030640040306401200FE0010030640000206400402064015120000880E0640480F0640080F0640C80F0640AB
:40118000880F0640D1010020B8010020B0010020BC010020D00100200023044A1360044A13601022034B1A707047C046680006406C000640D101002010B50E4A13685B0037
:4011C0005B08136000230C490B600C490B600C4804680C49214001600B490B600B490B6010210B4B19701368802109060B43136010BDC04600000640680006406C000640AC
:4012000060000640FF5CFFFF880F0640C80F0640D101002010B5C94B1B68002B00D09847C74B1B68DB0702D50022C64B1A60C64B1B789B0622D4C54B1A680223FF331A4212
:401240001CD0C14B1B78DB070AD5C14A137802218B431370117809230B43DBB213700AE0BB4A137820218B431370117870235B420B43DBB213700022B34B1A70B24B1B78A8
:401280009B0600D559E1B04B1B78DB0600D452E1AE4B1B689B0740D50222AE4B1A60AE490B680D321A40096880231B020B4000D001239B18A94A1278D2B2934206D2A44A7C
:4012C000117804230B43DBB2137006E0A34A12789B1AA3490A68D31A0B60A14B1A68A14B1A600023A04A13609C4A13709F4B1A68802149020A431A6019689D4A0A401A6010
:40130000934A137802218B431370117801230B43DBB2137010228C4B1A708C4B1B681B0739D508228B4B1A60924B1B689B040CD414E0914B1A68914909688A1890490968C7
:40134000C9B211701A6801321A608E4B1B681B07EFD1884A11688C4B0B4013608B4B1B689B0605D57A4A117840230B43DBB213700022874B1A60874A844B1A60744A137871
:4013800020218B431370117810230B43DBB213706D4B10221A706D4B1B685B0648D501227D4B1A607D4B1B68DB0610D50F326E4B1A606C4B1A686A4B1A60654A11780223A5
:4013C0000B43DBB2137012225F4B1A7025E0744B1B68694A12689B1A072B03D804226C4B1A6011E0082B06D1624A1368A02109020B43136008E05F4A1368802189010B4366
:4014000013600822624B1A60514A117820230B43DBB2137011224C4B1A70624A4D4B1A60614A116808230B43136001225F4B1A605F4B1B681B072AD5594B1B684E4A106835
:40144000181A0838082802D9002408200EE001240CE0494B1A68494909688A1848490968C9B211701A6801321A6001380028F0D1002C08D03F4A1368802109020B43136025
:401480000022434B1A600822404B1A6024E0484B1B685B0720D53A4B1B68374A1168404A126891420DD20121404A1160324A1168324800684118DBB20B7013680133136033
:4014C00007E0FFF7E9FD224A117840230B43DBB2137004222D4B1A60364B1B68DB0620D42BE01F4B1A68344B1B689A420CD21C4B1A68324909688A181278D2B230490A6067
:401500001A6801321A600CE0FF222D4B1A60134B1B78DBB20A2B04D8104A13780133DBB213700D4B1B680F221340082BD9D10132244B1A6001E0FFF73FFE10BDAC010020BF
:401540008C0E0640880E0640D10100204C0F0640B8010020400F064008020640D0010020B4010020B0010020880F064004020640FFFFFEFF60000640BC010020C801002037
:401580004003064008030640FF5FFFFFC00F0640C80F0640ED0F0000800E064064000640C4010020FF0F0000480F06406C000640CC0F06408C0F0640C0010020CC01002037
:4015C00040020640800F0640014B18687047C046F00000200E4B70B500251E000D4CE41AA410A54204D0AB00F35898470135F8E700F064F8084B00251E00084CE41AA4109C
:40160000A54204D0AB00F35898470135F8E770BDC8160000C8160000C8160000D0160000002310B59A4203D0CC5CC4540133F9E710BD03008218934202D019700133FAE7BE
:401640007047000080170000310000000000000090030000CE020000E0020000F00200000003000010030000200300004003000030030000500300006003000070030000DC
:401680008003000084050000A405000080070000F005000090060000800700009C060000C8060000F0050000EA060000620700009A11440A003C010143000000F8B5C046F1
:4016C000F8BC08BC9E46704729010000C5010000F8B5C046F8BC08BC9E46704701010000F01600007000002088000000E00000000000000044160000481600000100000068
:4017000000007017E02E00000C000000001BB7000000000000000000000000000000000000000000000000000000000000000000B816000000000000000000000000000068
:4017400000000000000000000000000000000000000000000000000000000000000000000000000000000000000000000000000090000020000000000000000000000000B9
:401780000000000000000000000000000000000000000000000000000000000000000000000000000000000000000000000000000000000000000000000000000000000029
:4017C00000000000000000000000000000000000000000000000000000000000000000000000000000000000000000000000000000000000000000000000000000000000E9
:4018000000000000000000000000000000000000000000000000000000000000000000000000000000000000000000000000000000000000000000000000000000000000A8
:401840000000000000000000000000000000000000000000000000000000000000000000000000000000000000000000000000000000000000000000000000000000000068
:403FC00000000000000000000000000000000000000000000100000000000000000000000000000000000000000000000000000000000000000000000000000000000000C0
:0200000490303A
:020000000E6090
:0200000490402A
:200000000000000000000000000000000000000000000000000000000000000000000000E0
:0200000490501A
:0C00000000020A44119A00010A4B1FFA8A
:0200000490600A
:0100000001FE
:00000001FF
